:100000000C943A000C9457000C9457000C94570031
:100010000C9457000C9457000C9457000C94570004
:100020000C9457000C9457000C9457000C945700F4
:100030000C9457000C9457000C9457000C945700E4
:100040000C9457000C9457000C9457000C945700D4
:100050000C9457000C9457000C9457000C945700C4
:100060000C9457000C9457000C9457000C945700B4
:100070000C94570011241FBECFEFD2E0DEBFCDBFDE
:1000800011E0A0E0B1E0E0E4F1E002C005900D92E3
:10009000A030B107D9F711E0A0E0B1E001C01D9296
:1000A000A030B107E1F70E9473000C949F000C94FC
:1000B0000000CF93DF93CDB7DEB7E5E2F0E010822A
:1000C000E4E2F0E01082E8E2F0E01082E7E2F0E043
:1000D0001082EBE2F0E01082EAE2F0E080E180835F
:1000E000DF91CF910895CF93DF93CDB7DEB70E9414
:1000F0005900A895E4E5F0E087EF8083E0E6F0E0C2
:1001000088E18083E0E6F0E01082E2E6F0E0108231
:1001100000C0E9E2F0E08081882344F0ABE2B0E087
:10012000EBE2F0E0808180618C93F3CFABE2B0E052
:10013000EBE2F0E090818FEE89238C93EACFFFCF42
:00000001FF
